:10000000025FB13200000000000000025CD6000078
:10001000000000320000000000000032000000007C
:100020000000000232780000000000025DC70000FE
:100030005052343032207665722E3131302E3520D8
:100040004864773A482034303030752032392D30CA
:10005000352D30342031323A343220202843295291
:100060006F6765722053702E4A2E207777772E7235
:100070006F6765722E706C2C2074656C2F666178CA
:10008000202B34382035352032373230313332208E
:100090002843296A502D706C2C204D6F6E61204CC6
:1000A0006973612043452C2049534F393030312C3E
:1000B0002031737420436C617373D320202052204D
:1000C00045205320452054D25052333032204C43E7
:1000D0004420763131302E35002D2D2F2D2D202D21
:1000E0002D3A2D2D004350523A20004C6F633A2098
:1000F000004C4F433A2000D22020202020202020F6
:100100002020202020202020D200454E545259206B
:10011000202000455849542020202000445554599F
:10012000204558495400494E5445524E414C00D147
:1001300020202020202020202020202020202020BF
:10014000D1435243202020204520722072206F206E
:10015000720020202020200020D1466C617368208E
:10016000435243204572726F722000D3436F6E6614
:100170006967204D656D204572726F7200D3205300
:10018000657276696365204F4E00D32053657276A1
:10019000696365204F464600D2204D415354455275
:1001A000204944203D20203F2000D3536574207413
:1001B000696D652048484D4D202020D200D35365FD
:1001C00074206461746520524D4D44445720D20020
:1001D000D22020202020202020202020202020206D
:1001E00020D2D501055245473A200000D3D5021050
:1001F00044206F2077206E206C206F2061206420C7
:1002000000D120202020202020202020202020205D
:10021000202020D1D5030C50617373776F72643F37
:10022000203A2000D2D50410204163636573732007
:1002300064656E696564202000D2D5051020416395
:1002400063657373206772616E7465642000D1D535
:100250000410204163636573732064656E6965648F
:100260002020D2D50610204E6F204475616C2045A9
:100270006E747279202000D3D509104475616C200A
:10028000456E747279204D6F64652000D1D50A0ADD
:100290002020204572726F72202300202020200031
:1002A000D1D50C1020202041504220526573657436
:1002B0002020202000D2D50E104C696D6974206575
:1002C00078636565646564202000D50F0C4E4F523D
:1002D0004D414C20202020202000D1D5041020208A
:1002E0004143434553532044454E59202020D2D505
:1002F0001010204150422056696F6C6174696F6E16
:10030000202000D1D50D10202020204964656E7476
:10031000204F4B20202020D2D510102041504220C9
:1003200056696F6C6174696F6E202000D2D5111010
:10033000204E6F206F6E6520696E736964652020A2
:1003400000D1D51210202020557365722049442019
:100350003D203F202000D320202020552053204541
:100360002052D2D51610202050726F6772616D6DC9
:10037000696E6700D3202020494E5354414C4C45B0
:100380005220202020D2D51610202050726F677284
:10039000616D6D696E6720202000D22020202046EC
:1003A000205220452045202020202000D22020203F
:1003B0004520582049205320542053202000D1D5D7
:1003C000041020204143434553532044454E5920B7
:1003D0002020D2D506102020496E70757420426C02
:1003E0006F636B73202000D1D5041020204143435C
:1003F0004553532044454E59202020D2D507102084
:1004000020434C4F534544204D4F4445202020006D
:10041000D1D5041020204143434553532044454E39
:1004200059202020D2D508104F7574206F66207493
:10043000696D65207A6F6E6500D1D504102020416A
:1004400043434553532044454E59202020D2D50BD9
:1004500010204F464620636F6E646974696F6E208A
:100460002000D1D51310202053574954434820442D
:10047000454E59202020D2D508104F7574206F6644
:100480002074696D65207A6F6E6500D1D5041020E7
:10049000204143434553532044454E59202020D208
:1004A000D5141020202020505245414C41524D205F
:1004B00020202000D1D5151020537769746368651A
:1004C000722049443D203F2000C28E53890F43894A
:1004D00010758BD6758D97C28FD28E308FFDC28EE0
:1004E00022C28E53890F438910758BEB758DCBC259
:1004F0008FD28E308FFDC28E22C28E53890F4389D8
:1005000010E58AC4242BF58B758DEBC28FD28E300B
:100510008FFDC28E22F9C3137004A253801814C039
:10052000E0030303540F2443F8D0E0540704F5F02C
:10053000E213D5F0FCE992E02275F0061205E922FB
:10054000C2A075F0061205E9D2A0221205401205DC
:1005500039120540120539120540120539120540BD
:1005600012053912054075F0181205E922C2A0756E
:10057000F04B1205E9D2A022755A0412323DC2A0F6
:1005800075F0C81205E9D2A022755A0512323D1243
:10059000056D75F01E1205E912056D22755A0712D8
:1005A000323D12055722755A0612323D12055D2260
:1005B00012054B12054B22755A0712323D755A0629
:1005C00012323D12055D12055D12055D22C2A1C207
:1005D0006812054075F0121205E9D2A1C268221214
:1005E000054075F0121205E9221204C9201E07C049
:1005F000F0122472D0F0D5F0F0227004A253B3228E
:10060000C0E014120609D0E022C0E0030303540F37
:1006100028F8D0E0C0E0540704F5F0E213D5F0FC70
:10062000D0E02212054B75F0641204C9D5F0FA220D
:1006300012055775F0C81204C9D5F0FA80F22230BD
:100640001716C217C2AC1204F91204F9D299120794
:1006500025C260D2B6125DD2301116C211C2AC12E0
:1006600004F91204F9D299121458C260D2B6125D7C
:10067000D2301316C213C2AC1204F91204F9D29983
:100680001214DDC260D2B6125DD2301216C212C28E
:10069000AC1204F91204F9D299121379C260D2B6DD
:1006A000125DD2301416C214C2AC1204F91204F94D
:1006B000D2991213BBC260D2B6125DD2301516C2E7
:1006C00015C2AC1204F91204F9D299121525C260B0
:1006D000D2B6125DD2301616C216C2AC1204F9128E
:1006E00004F9D2991215B8C260D2B6125DD2301890
:1006F00016C218C2AC1204F91204F9D299125A594E
:10070000C260D2B6125DD2E57A6013B40105122C34
:10071000828008B40205122C918000757A001224A0
:100720007212592422125C2CC2B67537007403125F
:100730003E60E51E123E60E51F123E607450123EA0
:1007400060747D123E60900000E535600F9003E814
:100750001460099007D0146003900BB87E7D7F0869
:1007600075F000C0F0125C27B40203D38001C3D03F
:10077000E033F5F0A3DFEC123E60DEE2E537123E37
:10078000603099FD22C0F075F0DCD5F005B2B512ED
:1007900055C7C0F01209CFD0F030E7EED0F022AA52
:1007A000F0120785E532652FF5F0E533653045F049
:1007B000600C1208F6852F32853033120785120936
:1007C000941207851209BC1207851209038AF022C8
:1007D000AAF0120785E532652FF5F0E5336530455F
:1007E000F0600C1208F6852F32853033120785121F
:1007F00009801207851209BC1207851209038AF0C5
:10080000227920752F017530037531E09000811237
:1008100007851208F61207851209547900752F0111
:100820007530047531009000A11207851208F61288
:10083000078512095479E0752F017530057531006F
:100840009001A11207851208F61207851209548536
:100850002F3285303322AAF0120785E532652FF555
:10086000F0E533653045F0600C1208F6852F3285CF
:10087000303312078512093C8AF022AAF01207854C
:10088000E532652FF5F0E533653045F0600C120870
:10089000F6852F328530331207851209248AF0221B
:1008A000C0F075F00833C297928300D297D5F0F567
:1008B000D0F022C0F075F008C297D29700A2823320
:1008C000D5F0F5D0F022D2B7D297D283D282D2849B
:1008D00022E53033E52F3322C3E5303322E53122E0
:1008E0001208A01208D11208A01208D81208A012EB
:1008F00008DD1208A0221208C6C28474531208E050
:10090000D284221208C6C28474581208E0D284220B
:100910001208C6C28474541208E0E41208A0120837
:10092000B3D284221208C6C28474541208E0E412BE
:1009300008A01208B3F608D9F9D284221208C6C258
:100940008474541208E0E41208A01208B3F208D923
:10095000F9D284221208C6C28474541208E0E41248
:1009600008A01208B3F0A3D9F9D284221208C6C095
:10097000E0C28474841208E0D0E01208A0D284227D
:100980001208C6C28474841208E0E61208A008D9CE
:10099000F9D284221208C6C28474841208E0E212DA
:1009A00008A008D9F9D284221208C6C2847484121D
:1009B00008E0E01208A0A3D9F9D284221208C6C226
:1009C0008474831208E0D2841204C91204C922C2BA
:1009D0008474571208A01208B3D28422D283D28220
:1009E000D297D2B7D284B2B575F0021204C9D5F04D
:1009F000FAC2B7B2B575F0021204C9D5F0FAD2B78F
:100A0000B2B522752F017530DB75310012078512E2
:100A10000C9E7532FF7533FF22AE83AD8290DB00F2
:100A20007F207404F9747CF8752F018583308582EA
:100A30003112087B787CE66E702508E66D70200820
:100A4000E6601AB4FF028013167404F9747CF8751A
:100A50002F018583308582311207D0C322D322A390
:100A6000A3A3A3DFBD80F490DB007F207404F9749E
:100A70007CF8752F0185833085823112087B787C64
:100A8000E66E700908E66D700408E6FC22A3A3A3D5
:100A9000A3DF0A7CFF2290DB007F207BFF7404F938
:100AA000747CF8752F0185833085823112087B783C
:100AB0007CE66E702C08E66D702708ECB4FF0D78AC
:100AC0007C76FF0876FF0876FF0874FFF67404F959
:100AD000747CF8752F018583308582311207D0C36D
:100AE00022BBFF10787CE6B4FF0A08E6B4FF05C31A
:100AF00074209FFBA3A3A3A3DFA3BBFF02D322EB1E
:100B0000232354FC2400F5827583DB50020583788F
:100B10007CEEF608EDF608ECF608E4F67404F974D9
:100B20007CF8752F018583308582311207D0C3226E
:100B300075830075F08E752F02858330753100C086
:100B4000F0C083120785120C9ED0830583D0F0D5A8
:100B5000F0E475830075F0DA752F03858330753105
:100B600000C0F0C083120785120C9ED0830583D08D
:100B7000F0D5F0E47532FF7533FF2275830075827E
:100B80000075F08EC0F0C082C083752F028583305F
:100B90007531001207851208F6D083D082C082C05A
:100BA00083752F008582307531001207851209BCCC
:100BB000D083D08205830582D0F0D5F0C77583003D
:100BC00075820075F0DAC0F0C082C083752F03858E
:100BD00083307531001207851208F6D083D082C0A9
:100BE00082C083752F01858230753100120785120E
:100BF00009BCD083D08205830582D0F0D5F0C775BB
:100C000032FF7533FF2275830075820075F08EC048
:100C1000F0C082C083752F008583307531001207C4
:100C2000851208F6D083D082C082C083752F0285DA
:100C300082307531001207851209BCD083D082053D
:100C4000830582D0F0D5F0C775830075820075F0FA
:100C5000DAC0F0C082C083752F0185833075310002
:100C60001207851208F6D083D082C082C083752F08
:100C7000038582307531001207851209BCD083D0FC
:100C80008205830582D0F0D5F0C77532FF7533FF3A
:100C9000221208C6C28474501208E0D284221208BC
:100CA000C6C28474811208E0D284221208C6C284AB
:100CB00074841208E0E81208A0D9FAD28422AAF0BB
:100CC000120785E532652FF5F0E533653045F060B4
:100CD0000C1208F6852F32853033120785120CABC3
:100CE0001207851209BC8AF0221208C6C284745405
:100CF0001208E0E41208A0E4C0E01208B3D0F02526
:100D0000F0D9F5D28422758300758202800675833E
:100D100000758200E475F08D85822F8583307531F2
:100D200000C082C083C0F0C0E01207851208F6122E
:100D300007857900120CE9D0F025F0D0F0D083D0EF
:100D4000820583D5F0D285822F858330753100C02E
:100D5000E01207851208F61207857920120CE9D0F7
:100D6000F025F07532FF7533FF227583007582031D
:100D70008006758300758201E475F0DA85822F851F
:100D80008330753100C082C083C0F0C0E012078597
:100D90001208F61207857900120CE9D0F025F0D080
:100DA000F0D083D0820583D5F0D27532FF7533FF42
:100DB00005E02275830075F000752F00858330757E
:100DC0003100C0F0C083120785120C9ED0830583CA
:100DD000D0F0D5F0E47532FF7533FF75830075F000
:100DE000DA752F01858330753100C0F0C08312079A
:100DF00085120C9ED0830583D0F0D5F0E47532FFC8
:100E00007533FF221205637555FA3090FA75F005B7
:100E10001204C9D5F0FA7555FA2090FA22E577B494
:100E200006FAE5831252DEE5821252DE7800E21203
:100E300052DE7801E21252DE7802E21252DE120E27
:100E40000422C0E0E577B40928D0E0787CE61252AD
:100E5000DE08E61252DE08E61252DE08E61252DE24
:100E600008E61252DE08E61252DED2AF120E04C0BD
:100E7000E0D0E022E577B4053DED600F1414600B7F
:100E8000146008146005ED2488502BE583C082129D
:100E900052DED082E5821252DEED1252DE787CE61E
:100EA0001252DE08E61252DE08E61252DE08E612A0
:100EB00052DE08120E042222E577B405F9ED2488EB
:100EC00050F4C082C083787CE60354012430E612DB
:100ED00052DE08E61252DED083D082E583C082C0A3
:100EE000831252DED083D082E582C082C083125248
:100EF000DE120E04D083D0822222E577B4050FEDF6
:100F00002488500A74303073027431120E04223077
:100F100008597881E6540FC0E0E6C4540375F00A1E
:100F2000A4D0F025F0FD7882E630E402240A540FC4
:100F3000FE901A007F3C7404F97400F8752F018547
:100F400083308582311208567800E26D701708E20E
:100F50006E701208E2C42354E0F5F07882E6541F64
:100F600045F0F68006A3A3A3A3DFCB221261CA1229
:100F70000F0F1261D9FEAFF01257147DFF0DED3047
:100F8000E70122D27375F004A42481F582E5F034E0
:100F900000F583C082C083787CE0F6A308E0F6A366
:100FA00008E0F6A308E0F6D083D082120E74787CB5
:100FB0008683088682787CB6FF0708B6FF03021096
:100FC00025C3E58233F582E58333F583E58224E0AA
:100FD000F582E5833405F583787EE6704808E6609F
:100FE00044FB7402F9747CF8752F01858330858287
:100FF0003112087B120EB7A3A3787CE60856B4FF23
:1010000003021025787C86F053F07F08E6C39EC06B
:10101000E0E5F09FD0F0400445F07009787CE6A24E
:10102000E79273DBBD120EF9BD003DB273122C10B6
:101030004033203C30201F0E303D0B2052053073D2
:1010400024800320731FA273925292E0A25392E174
:10105000F5F013925365F030E00B205305122CA0ED
:101060008003122CAF020F7DED14C0E00303035484
:101070000F2443F8D0E0540704FB7400D333DBFDA6
:10108000307305FBE24B8004F4FBE25BF2020F7D60
:101090001208A01208D11208A01208D8D2E0120833
:1010A000A01208DD1208A0221208C6C284745412CD
:1010B0001090E41208A01208B3F608D9F9D28422DD
:1010C0001208C6C2847484121090E61208A008D9CF
:1010D000F9D2842290FC00752F0475300075310020
:1010E000C082C0837555FA1207851208F6852F79DC
:1010F0008530787908787C1207851210A81212D0F2
:10110000D083D0827044C082C08378808683088672
:10111000821211814024787E868308868212118192
:1011200040181211A0E582600AE575B5780CE576E5
:10113000B57907D083D08202115C787EE6249AF6D6
:10114000121313125284D083D0820530E53070021E
:10115000052FA3E582458370871211637532FF75F1
:1011600033FF22787E760008760078807600087655
:10117000000876000876007579047578001212EF81
:1011800022C082C083E5822400F582E5833480F5A5
:10119000834005D083D08222D083D0829000002269
:1011A000E58275F008A4F582E5F0C58375F008A422
:1011B0002583F583E5F03404F576E5822400F58295
:1011C000E5833400F583500205768583752212523B
:1011D00094D083D08222C082C0831212A970EF788B
:1011E0007E868308868212118140E31211A01216B6
:1011F0001D787C76007880E518F608E519F6087603
:10120000000876007408F9747CF885762F858330A1
:101210008582311207D07404F97480F885762F85A1
:10122000833085823112087B75F004787C7980E602
:1012300067600280990809D5F0F51212B0787E86B1
:1012400083088682A3121181787EA68308A68278FD
:10125000808683088682121181787EE66583700A13
:1012600008E665827004A31211817880A68308A61F
:1012700082C079C0788576798575781212EFD0E0D2
:10128000D0F0B57809C5F0B579028018C5F0C079FD
:10129000C07885F079F578787EE62499F6121313F4
:1012A000D078D079D083D082221212B01212D022FC
:1012B00085792F8578307531001207851208F67907
:1012C00008787C1207851210A8852F3285303322CA
:1012D0007881E618261826182618245566700F7887
:1012E00081E61866186618661866186499662212F0
:1012F00012F6121313227881E618261826182618DB
:101300002455F67881E6186618661866186618641B
:1013100099F62285792F857830753100120785126C
:1013200008F61207857908787C1210C0120785121A
:1013300009BC120785120903852F3285303322122A
:1013400012A97030787EE6C0E008E6C0E008868327
:10135000088682C3D0E09582F582D0E09583F5833C
:1013600050104582600CE5822400F582E5833480CC
:10137000F583C322900000D322C2B612133FE43398
:10138000C0E07537007403123E60E51E123E60E552
:101390001F123E607453123E60D0E0123E60740033
:1013A000123E607400123E60E583123E60E58212D8
:1013B0003E60E537123E603099FD22C2B6E53560E9
:1013C00004F4FF8004FF1211637537007403123EAA
:1013D00060E51E123E60E51F123E607456123E60CC
:1013E000EF123E60E537123E603099FD227401C075
:1013F000E0787C75F008E4F608D5F0FBD0E0D32265
:1014000012133F40E860E8788086830886821214D1
:1014100013C322C082C083E58275F008A4F582E57B
:10142000F0C58375F008A42583F583E5F03404F551
:1014300076E5822400F582E5833400F583500205C9
:10144000767408F9747CF885762F8583308582312F
:1014500012087BD083D0822212133F7F08500512DE
:1014600011637F00787E8663088664088665088637
:1014700066C2B67537007403123E60E51E123E6008
:10148000E51F123E607454123E60E535123E60EF77
:10149000123E60E535603CE5666564F5F0E565653E
:1014A0006345F0600B8566828565831214138003A3
:1014B0001213EF856682856583A31211818582668A
:1014C000858365787C75F008E6123E6008D5F0F8F3
:1014D000D535C4E537123E603099FDC322E535703D
:1014E00007C2AF12133F5005E535F4800C7880A693
:1014F0006508A6661212EFE535D2AFC0E0C2B67538
:1015000037007403123E60E51E123E60E51F123E76
:10151000607455123E60D0E0123E60E537123E60C6
:101520003099FDD322C2B61261CA75370074031216
:101530003E60E51E123E60E51F123E607457123E8B
:10154000607881E623235403123E607882E630E41B
:1015500002240A541F123E607881E6C45401F5F05B
:10156000A4E5F0E6540F25F0123E607881E6C454FD
:1015700001F5F0A4E5F0E6540F25F0123E60787F07
:10158000E6C45403F5F0A4E5F0E6540F25F0123E4E
:1015900060787EE6C45403F5F0A4E5F0E6540F2528
:1015A000F0123E607882E603C45407123E60E537CD
:1015B000123E603099FDD322C2B675370074031213
:1015C0003E60E51E123E60E51F123E607458123EFA
:1015D000607420232354FC04123E607420123E6089
:1015E00090DB007F207404F9747CF8752F018583EB
:1015F0003085823112087B787CE6123E6008E61264
:101600003E6008E6123E6008E6123E6008A3A3A30F
:10161000A3DFD2E537123E603099FDD3221261CAB2
:101620007882E630E402240A540FC4F97881E6C4D3
:10163000540375F00AA4F5F0E6540F25F0C31349DE
:10164000787DF67881E692E754C0F9787FE6C45455
:101650000775F00AA4F5F0E6540F25F049F97880F3
:10166000E6C4540375F00AA4F5F0E6540F25F0F52E
:10167000F0787EE654702345F0787FF6787EE9F6C0
:1016800022C082C083E52F1252DEE5301252DE788E
:101690007EE61252DE08E61252DE08E61252DE083C
:1016A000E61252DE120E04D083D0822253620F5310
:1016B000610F5318F053190FC2AFE5612324ADF841
:1016C000E5184519F608A61A056153610FE561B5DD
:1016D0006205056253620FD2AF22E562B5610574FF
:1016E00000780022C33324ADF8E6C0E008E6F8D065
:1016F000E022223054FDC2A075F0061205E9D2A006
:1017000075F0141205E9E545C25422301E037554E4
:10171000F01222A8205407740F301E0580F3121611
:10172000F322F5F00303543FB40267E53E6408601A
:1017300005E53EB40D59E5F089F0C0F030081CC055
:10174000E07877E26013C3335005D0E002176E12E1
:10175000051550F6D0E002175BD0E0D0F0A9F054A8
:1017600003B40211C231A231B392A5021861D0F0C4
:10177000A9F0021861B4010AD231A231B392A502D4
:101780001861B4030AB231A231B392A50218610202
:10179000185FB40365E53F64086005E53FB40DEFED
:1017A000E5F089F0C0F030081CC0E07878E2601302
:1017B000C3335005D0E00217D812051550F6D0E01B
:1017C0000217C5D0E0D0F0A9F05403B40211C23220
:1017D000A232B392A6021861D0F0A9F0021861B447
:1017E000010AD232A232B392A6021861B40309B23E
:1017F00032A232B392A680698065B40462E5406487
:10180000086005E540B40D57E5F089F0C0F03008F8
:101810001CC0E0787EE26013C3335005D0E00218AC
:101820003F12051550F6D0E002182DD0E0D0F0A9F7
:10183000F05403B4020FC237A237B392808022D093
:10184000F0A9F0801CB40109D237A237B39280808E
:1018500010B40309B237A237B3928080048000D35A
:1018600022C322787375F00EE4F208D5F0FB74FF02
:10187000787BF2787CF222D24E6F20657874656EA8
:10188000646564202020202020202000756FFF1236
:101890001863C208C207120D72602E20082A740154
:1018A000F9747CF8752F0075308C7531EE12087B59
:1018B000797CE7B4FF12C246C247C248C249C24A55
:1018C000C24BC24CC24DC24E221208017401F974BF
:1018D0006FF8752F017530037531A012087B740EF7
:1018E000F97473F8752F017530037531A11208561C
:1018F0007410F97453F8752F017530037531C012E7
:1019000008567410F97463F8752F0175300375313A
:10191000D0120856D208D20722797C774809774E30
:1019200009776E0977A07404F9747CF8752F007537
:10193000308D7531201207D07404F9747CF8752F3E
:101940000275308D7531201207D022E4A22492E076
:10195000A22592E1A22692E2797CF77401F9747CC7
:10196000F8752F0075308C7531E81207D02274019C
:10197000F9747CF8752F0075308C7531E812087B8E
:10198000797CE7A2E09224A2E19225A2E2922622AB
:10199000797CE4A23892E0A23992E1A23A92E2A2E2
:1019A0001C92E392E492E5A23C92E6A23D92E7F714
:1019B00009E4A23B92E0A23E92E1A23F92E2A24061
:1019C00092E3A24292E4A24392E5A24492E6A245A7
:1019D00092E7F709E4A24692E0A24792E1A2489278
:1019E000E2A24992E3A24A92E4A24B92E5A24C926F
:1019F000E6A24D92E7F7E4A24E92E0A20292E1A2A3
:101A00000392E2F77404F9747CF8752F0075308C3A
:101A10007531EC1207D0227404F9747CF8752F002C
:101A200075308C7531EC12087B797CE7A2E0923836
:101A3000A2E19239A2E2923AA2E3921CA2E6923C7F
:101A4000A2E7923D09E7A2E0923BA2E1923EA2E228
:101A5000923FA2E39240A2E49242A2E59243A2E620
:101A60009244A2E7924509E7A2E09246A2E192479A
:101A7000A2E29248A2E39249A2E4924AA2E5924BE2
:101A8000A2E6924CA2E7924D09E7A2E0924EA2E1B3
:101A90009202A2E2920322797CF77401F9747CF835
:101AA000752F0075308C7531E41207D0227401F95E
:101AB000747CF8752F0075308C7531E412087B79D1
:101AC0007CE7227401F97438F8752F0075308C7535
:101AD00031FC1207D0227401F97438F8752F0075A3
:101AE000308C7531FC12087B227401F97439F87559
:101AF0002F0075308D7531001207D0227401F974F2
:101B000039F8752F0075308D75310012087B2274FD
:101B100002F9743FF8752F0075308C7531FD12088D
:101B2000567402F97441F8752F0075308D753101C6
:101B3000120856227402F9743FF8752F0075308C24
:101B40007531FD12079F7402F97441F8752F007505
:101B5000308D75310112079F227401F9743AF875BE
:101B60002F0075308C7531F01207D07401F9743B79
:101B7000F8752F0075308C7531F41207D07401F9A7
:101B8000743CF8752F0075308C7531F61207D074DF
:101B900001F9743DF8752F0075308C7531F212071C
:101BA000D0227401F9743AF8752F0075308C7531B4
:101BB000F012087B7401F9743BF8752F0075308CB6
:101BC0007531F412087B7401F9743CF8752F0075B7
:101BD000308C7531F612087B7401F9743DF8752F5D
:101BE0000075308C7531F212087B227401F9743E55
:101BF000F8752F0075308C7531F81207D07401F923
:101C0000743FF8752F0075308C7531FA1207D07457
:101C100001F97440F8752F0075308C7531FB12078F
:101C2000D0227401F9743EF8752F0075308C75312F
:101C3000F812087B7401F9743FF8752F0075308C29
:101C40007531FA12087B7401F97440F8752F00752C
:101C5000308C7531FB12087B227402F9741EF87502
:101C60002F0075308C7531E01207D0227402F974A0
:101C70001EF8752F0075308C7531E012087B22C07C
:101C800082C083E58275F008A42420F58250020505
:101C9000F0A8F0E58375F008A4282400F583787C8B
:101CA00076FF7401F9747CF8752F00858330858286
:101CB000311207D0A3A3A3A3A37401F9747CF87510
:101CC0002F008583308582311207D0D083D082C225
:101CD00007220809E7C4F5F066540F700D08E7F510
:101CE000F066540F7004DAEAE422E6540FC5F054AB
:101CF0000FC395F09206740122788179277A03E662
:101D0000C4540FF309E6540FF30908DAF27927787F
:101D1000A07A06E6540FF6E36670080908DAF4E4E0
:101D2000C25A22792C78A57A06C3E3961918DAFAF2
:101D30009206792C78A57A06E3540FB40F08E6547E
:101D40000FB40F108008E6540FB40F0B800618195B
:101D5000DAE680CB740122C3E396B4090280121440
:101D6000600FC3E3F5F0E695F0B409028003147048
:101D7000E3E9B42704E4D25A221918E366540F6049
:101D8000F080D1121CF9701A305A17203B157518C3
:101D90005085831985821A1216AC7553B4D256D267
:101DA00059E42204227408F9747CF8752F00753008
:101DB0008C7531C012087B7894797C7A05121CD41A
:101DC000227408F9747CF8752F0075308C7531C059
:101DD00012087B121D83227405F9747CF8752F009C
:101DE00075308C7531C01207D0227403F97481F8F4
:101DF000752F0075308C7531C51207D022C082C096
:101E000083E5822420F582E583347DF5837401F92E
:101E10007441F8752F0085833085823112087BD09C
:101E200083D082C082C083E58275F008A42420F5A7
:101E300082500205F0A8F0E58375F008A42824007C
:101E4000F5837408F9747CF8752F008583308582DA
:101E50003112087BD083D08222C082C083E5827594
:101E6000F008A42420F582500205F0A8F0E583755F
:101E7000F008A4282400F5837408F97494F8752FE9
:101E80000085833085823112087BD083D08222C0C6
:101E900082C083E58275F008A42420F582500205F3
:101EA000F0A8F0E58375F008A4282400F5837406F3
:101EB000F9747CF8752F0085833085823112087B98
:101EC000D083D082227405F9747CF8752F007530A8
:101ED0000075312012087B7894797C7A05121CD425
:101EE00022751B20751C009000007405F9747CF8A5
:101EF000752F00851C30851B3112087B7894797C06
:101F00007A05121CD46018E51B2408F51B50020545
:101F10001CA3E583B40FD3E582B4A0CE74012212D2
:101F20001DFDE42220070280B8751B00751C00759A
:101F3000739F75740FE573251BC2E0F582E5743558
:101F40001CF583C082C083E5822400F582E58334DA
:101F50001BF5837402F9747CF8752F018583308535
:101F6000823112087B787C8683088682121DFD7878
:101F700094797C7A05121CD47005D0F0D0F022D070
:101F800083D082C3E58313F583E58213F5822006AF
:101F900014E58245836023E58224FFF573E58334ED
:101FA000FFF5748007A385821B85831CC3E57395A9
:101FB0001BE574951C4003021F35740122751B2517
:101FC000751C009000007403F97481F8752F00856A
:101FD0001C30851B3112087B121D836018E51B2401
:101FE00008F51B5002051CA3E583B40FD9E582B4A4
:101FF000A0D4740122121DFDE42278A0E6540FB48F
:102000000F0302209420070280B3751B00751C008B
:1020100075739F75740FE573251BC2E0F582E57437
:10202000351CF583C082C083E5822400F582E583F8
:10203000343BF5837402F9747CF8752F0185833085
:1020400085823112087B787C8683088682121DFD8A
:10205000121D837005D0F0D0F022D083D082C3E56A
:102060008313F583E58213F582200614E582458308
:102070006022E58224FFF573E58334FFF574800761
:10208000A385821B85831CC3E573951BE574951C92
:102090004002808274012278947A0579A8E6540F70
:1020A000C4F5F008E6540F45F0F70809DAEF22C24C
:1020B000A3C266C2A2C269C2A1C268D2B775F00249
:1020C0001204C9D5F0FA20B72BD21ED2A3C266C221
:1020D000A2D269D2A1C268D2A4C267120563B2B506
:1020E00075F00F1204C9D5F0FA30B7EF122168C2AB
:1020F000AF025F6AD2A0120D0E700712212F1218C4
:102100008C22C21E7555FA75F0641204C9D5F0FA16
:10211000C2A0C2A2C26975F0641204C9D5F0FAD295
:10212000A0D2A2C269D2B71204E130B79C80D31208
:10213000196E121A17121AADA2E0924FA2E1925034
:10214000A2E29251121AD6121AFC121BA2121C22DF
:10215000121B0F121C6C22C2A3C266C2A2C269C2A9
:10216000A1C268D2A4C26722D21E12514740E8C25F
:10217000A3C266C2A2C269C2A1C268D2A4C267C019
:102180001EC01F787C9000007A08E6F008A3DAFAF7
:102190001221BD787C9000007A08E0F608A3DAFAF4
:1021A000900000124B55121DD7121DEAD01FD01EF1
:1021B000121C59124BCF121163120A0322120DB3D3
:1021C000751E30751F30C224C225C226C238C239DE
:1021D000C23AC21CC23CC23DC23BD23EC23FC24018
:1021E000C242C243C244C245C246C247C248C249B3
:1021F000C24AC24BC24CC24DC24E783F7422F20852
:102200007400F278417406F2087400F2C24FC250B2
:10221000C251753804753909753A01753B02753C30
:1022200004753D04753E07753F00754000121C594A
:1022300012194B121990C2E0A24F92E0A25092E103
:10224000A25192E2121A97121AC3121AE9121B59DA
:10225000121BEB121B34C208C207121919125B12AF
:1022600022306B04C26B800975F00C20B205D5F0EA
:10227000FAD322C322122261502DE8C0E0E9C0E067
:10228000EAC0E0755A0075F0031204C9D5F0FA12DD
:1022900030CE75F0031204C9D5F0FA122F52D0E0F7
:1022A000FAD0E0F9D0E0F822D2638008C2631223AA
:1022B0001A754200C21DD26B7555FA7440301E0269
:1022C000740CF552C262C254E55260391222752074
:1022D000623375F0031204C9D5F0FA12063F201ECE
:1022E00003201D183054E120631B7552601216F351
:1022F000B40B0D75F0081204C9D5F0FAD26280054E
:1023000012230D80C3C261D2AF7555FA2253420722
:10231000F8E54224A0C8F605422278A075F00874BA
:10232000FFF608D5F0FB22306109202303D22322D7
:10233000C26122C22322D2638004D26BC263C21D57
:102340007555FAD2227440301E02740CF5521223D5
:102350001A754200C262C261C254C26512063F20B1
:102360001E03201D2112227520621D20611A305487
:10237000212063147552601216F3B40B1275F00825
:102380001204C9D5F0FAD2627555FA125714221206
:10239000230DE55260F21257143065FD80BC85387C
:1023A00056755700B230E5386002D230A230B39291
:1023B000A7D26B22301D012278A0760A087603800E
:1023C0000778A0760A0876010875F06484F608E5B7
:1023D000F075F00A84F608A6F0754205D21D227544
:1023E00018C0751900751A011216AC22755100C279
:1023F000587518C0751900751A021216AC22D256FB
:102400007553B475185075190F751AFF1216AC2252
:10241000C20A12239E20480C75181075190F751AE0
:10242000FF1216AC2220480C75182075190F751A6A
:10243000FF1216AC2275186075190F751AFF121667
:10244000AC2275187075190F751AFF1216AC22128E
:102450005B127518C0751900751A0E1216AC22128F
:1024600025B6400D1227B240081229624003122BF4
:102470004522301E03C38006A290302401B3783673
:10248000E233F2B4FF0280060225C002266C202748
:1024900003202DF7D22D30081CC0E07873E26013C2
:1024A000C3335005D0E002266C12051550F6D0E07B
:1024B0000224B5D0E0E53A60D2B40126D20B122353
:1024C000DF30301520460C755702755602304A032E
:1024D00075560185395102266C2044031223FE02F1
:1024E000266CB40215303903205309206D061224DE
:1024F0001002265E12242502266CB40308C2531271
:10250000243502266CB40705D277757B03B4090C19
:102510002053032045030225A802266CB40A027446
:102520003DB4340874001223B402266CB435087428
:10253000101223B402266CB4360874111223B402AC
:10254000266CB4370874201223B402266CB4381BEE
:102550007401F9747CF8752F0075308C7531F112A7
:10256000087B787CE61223B402266CB4391B740114
:10257000F9747CF8752F0075308C7531F112087B79
:10258000787CE61223C102266CB43C0612244F026A
:10259000265EB43D13205308D25312244202265E15
:1025A000C25312243502265E751890751909F51A62
:1025B0001216AC02266CE53AB40B03A22D22C322FC
:1025C00070F1202703302DEBC22D30081CC0E078BD
:1025D00073E26013C3335005D0E002266C12051578
:1025E00050F6D0E00225E9D0E0E53A6022B40107D8
:1025F000C20B1223EC8075B402028070B40307D2C0
:10260000531224428066B409082053443045418067
:102610005BB40A02743DB432028051B43302804C80
:10262000B4340302266CB4350302266CB4360302BC
:10263000266CB4370302266CB4380302266CB43916
:102640000302266CB43C0302266CB43D0302266CE4
:102650007518A0751909F51A1216AC02266C10042B
:102660000302266C12576F12059CD204C227301E3B
:1026700003C38006A291302501B37837E233F2B468
:10268000FF0280060227BC022868202803202EF7BC
:10269000D22E30081CC0E07874E26013C3335005BA
:1026A000D0E002286812051550F6D0E00226B1D01D
:1026B000E0E53B60D2B40126D20B1223DF303015A7
:1026C00020460C755702755602304A03755601852F
:1026D00039510228682044031223FE022868B402FC
:1026E00015303903205309206D0612241002285A90
:1026F000122425022868B40308C253122435022884
:1027000068B40705D277757B03B4090C2053032006
:1027100045030227A4022868B40A02743DB43408B1
:1027200074001223B4022868B4350874101223B45C
:10273000022868B4360874111223B4022868B4372A
:102740000874201223B4022868B4381B7401F97489
:102750007CF8752F0075308C7531F512087B787C0C
:10276000E61223B4022868B4391B7401F9747CF8AA
:10277000752F0075308C7531F512087B787CE61268
:1027800023C1022868B43C0612244F02285AB43DE3
:1027900013205308D25312244202285AC25312243F
:1027A0003502285A75189075190AF51A1216AC02D6
:1027B0002868E53BB40B03A22E22C32270F1202827
:1027C00003302EEBC22E30081CC0E07874E2601398
:1027D000C3335005D0E002286812051550F6D0E04A
:1027E0000227E5D0E0E53B6022B40107C20B1223CB
:1027F000EC8075B402028070B40307D253122442F5
:102800008066B40908205344304541805BB40A0215
:10281000743DB432028051B43302804CB4340302AC
:102820002868B43503022868B43603022868B43730
:1028300003022868B43803022868B4390302286800
:10284000B43C03022868B43D030228687518A075DB
:10285000190AF51A1216AC02286810040302286837
:1028600012576F12059CD204C228301E03C3800683
:10287000A292302601B37838E233F2B4FF02800628
:1028800002296C0229FF202903202FF7D22F3008BC
:102890001CC0E07875E26013C3335005D0E0022914
:1028A000FF12051550F6D0E00228ADD0E0E53C60FF
:1028B000D2B40705D277757B03B4090C20530320EB
:1028C00045030229540229FFB40A02743DB43408B6
:1028D00074001223B40229FFB4350874101223B413
:1028E0000229FFB4360874111223B40229FFB43749
:1028F0000874201223B40229FFB4381B7401F97440
:102900007CF8752F0075308C7531F712087B787C58
:10291000E61223B40229FFB4391B7401F9747CF860
:10292000752F0075308C7531F712087B787CE612B4
:1029300023C10229FFB43C0612244F0229F1B43D01
:1029400013205308D2531224420229F1C2531224F5
:10295000350229F175189075190CF51A1216AC028A
:1029600029FFE53CB40B03A22F22C32270F12029DA
:1029700003302FEBC22F30081CC0E07875E26013E3
:10298000C3335005D0E00229FF12051550F6D0E000
:10299000022995D0E0E53C6009B409082053443091
:1029A0004541805BB40A02743DB432028051B433B5
:1029B00002804CB434030229FFB435030229FFB46A
:1029C00036030229FFB437030229FFB43803022972
:1029D000FFB439030229FFB43C030229FFB43D03CD
:1029E0000229FF7518A075190CF51A1216AC0229E8
:1029F000FF1004030229FF12576F12059CD204C274
:102A000029301E03C38006A285303301B37839E232
:102A100033F2B4FF028006022B4F022BFB2034035B
:102A20002036F7D23630081CC0E0787DE26013C350
:102A3000335005D0E0022BFB12051550F6D0E00212
:102A40002A44D0E0E53D60D2B40126D20B1223DF48
:102A500030301520460C755702755602304A037502
:102A60005601853951022BFB2044031223FE022B11
:102A7000FBB40215303903205309206D06122410CF
:102A8000022BED122425022BFBB40308C25312249F
:102A900035022BFBB40705D277757B03B4090C20F4
:102AA0005303204503022B37022BFBB40A02743D6B
:102AB000B4340874001223B4022BFBB4350874102C
:102AC0001223B4022BFBB4360874111223B4022B68
:102AD000FBB4370874201223B4022BFBB4381B74E8
:102AE00001F9747CF8752F0075308C7531F312087C
:102AF0007B787CE61223B4022BFBB4391B7401F9FA
:102B0000747CF8752F0075308C7531F312087B7862
:102B10007CE61223C1022BFBB43C0612244F022B8D
:102B2000EDB43D13205308D253122442022BEDC2C0
:102B300053122435022BED75189075190DF51A12E4
:102B400016AC022BFBE53DB40B03A23622C3227068
:102B5000F12034033036EBC23630081CC0E0787DFB
:102B6000E26013C3335005D0E0022BFB1205155071
:102B7000F6D0E0022B78D0E0E53D6022B40107C238
:102B80000B1223EC8075B402028070B40307D25399
:102B90001224428066B40908205344304541805BCA
:102BA000B40A02743DB432028051B43302804CB492
:102BB0003403022BFBB43503022BFBB43603022B88
:102BC000FBB43703022BFBB43803022BFBB43903ED
:102BD000022BFBB43C03022BFBB43D03022BFB7521
:102BE00018A075190DF51A1216AC022BFB10040370
:102BF000022BFB12576F12059CD204C234205B01DA
:102C000022C25B751840751900751A001216AC22A5
:102C1000E53A64036008E53B64036002C322D32203
:102C20001205DF30080C125360400390FFF112537D
:102C3000A522C05B122C50D05B22300813125360C7
:102C4000400390FFF11253A55005F55B1253FC228F
:102C5000E55B7005755B108023B41005755B118012
:102C60001BB41105755B208013B42005755BFF80D4
:102C70000BB4FF05755B008003755BFF125463E5C1
:102C80005B22C25375186075190F751AFA1216ACCB
:102C900022D25375187075190F751AFA1216AC22D4
:102CA000C25375186075190F751AE01216AC22D24E
:102CB0005375187075190F751AE01216AC22122D83
:102CC000B2122E49122EE022122DBF122E56122EB3
:102CD000ED22B20C30081CC0E07877E26013C333F9
:102CE0005005D0E0022D3512051550F6D0E0022C2B
:102CF000F3D0E0E53E604C24F84005E53E022D4E61
:102D0000E53EB40904A209803DB40A04A20B803652
:102D1000B40C03D38030B40D0B302B03022DCCD276
:102D20002BD38022B40E04A20A801BB40F04A27716
:102D30008014022DCCB40D06202B03022DCCC22B07
:102D4000C38003A253B39231B392A5022DCC300CB1
:102D50005E5359037859A2E282564030A2E082576E
:102D60004012A2E182584018C231A231B392A57636
:102D700000022DCCB60102801D76017558408016E8
:102D8000B60202801176027558A0800AB60302804E
:102D90000576037558CCE55823F55820E00AC23172
:102DA000A231B392A5022DCCD231A231B392A502A9
:102DB0002DCCE53EB40B07D231A231B392A522E56A
:102DC0003EB40B07C231A231B392A52230081CC019
:102DD000E07878E26013C3335005D0E0022E2D1264
:102DE000051550F6D0E0022DEBD0E0E53F604C2415
:102DF000F84005E53F022E46E53FB40904A20980EC
:102E00003DB40A04A20B8036B40C03D38030B40D59
:102E10000B302C03022E63D22CD38022B40E04A2DA
:102E20000A801BB40F04A2778014022E63B40D062F
:102E3000202C03022E63C22CC38003A253B3923210
:102E4000B392A6022E63022E63E53FB40B07D23283
:102E5000A232B392A622E53FB40B07C232A232B32C
:102E600092A62230081CC0E0787EE26013C3335083
:102E700005D0E0022EC412051550F6D0E0022E82D5
:102E8000D0E0E540604C24F84005E540022EDDE549
:102E900040B40904A209803DB40A04A20B8036B4F0
:102EA0000C03D38030B40D0B303503022EFAD2352B
:102EB000D38022B40E04A20A801BB40F04A2778030
:102EC00014022EFAB40D06203503022EFAC235C3C1
:102ED0008003A253B39237B39280022EFA022EFAE5
:102EE000E540B40B07D237A237B3928022E540B455
:102EF0000B07C237A237B392802222C0F075F0FAD6
:102F0000D5F0FD75F064D5F0FDD0F022122EFB1245
:102F10002EFB122EFB122EFB122EFB122EFB227505
:102F20006908A2E7B392B4C293122EFBC2B4D29343
:102F3000122EFBC0E0E430B201040030B201040004
:102F400030B20104D36003D5E001C3D0E033D569CA
:102F5000D122D293C2B4D2B2122EFBC293122F0C42
:102F6000D293122F0C204C06201E0330722B788C2B
:102F70007601087480F608A2A3B392E4304C027480
:102F8000B3F6748008304C0274B0F608304C02740A
:102F900080F608F608F6022FDC788C760308768037
:102FA000087480A26692E5A2A3B392E4201E0B20CF
:102FB0007208A26992E1A23092E0F6087480201EA5
:102FC0001220720FE55A54074480A26892E5A2A12C
:102FD000B392E4F6087480F608F608F675F0077800
:102FE0008C7E007F00E62EFEE6122F1FF62FFF08D4
:102FF000D5F0F2EED333122F1FF8EFD3336870629F
:10300000788CB6FF5D056BE56B24FE5014756B0282
:1030100020200ED2207518C0751900751A031216DB
:10302000AC204C06201E033072030230B77892E6C3
:1030300020E35720E24720E17E788DE6B60078084D
:10304000B64274D277757B037518B0751900751A7E
:10305000001216AC7518C0751900751A071216AC57
:103060008055E56B6014D56B1130200EC2207518A9
:10307000C0751900751A041216AC0230B7788D8627
:103080004208D26279A07A048008788DD26179945E
:103090007A05D27175F00FE6C4540FF755F0F5F0CC
:1030A00009E6540FF755F0F5F00908DAEAE5F0B44F
:1030B0000F051977EEC261D293C2B475F005120400
:1030C000E120B2061204E130B203D5F0F122D2932E
:1030D000C2B4D2B2122EFBC293122F0CD293122F73
:1030E0000C201E1F307123788C7611748008F6082E
:1030F000A2A3B392E4F6748008F608F608F608F680
:10310000023150788C761502310E788C7613087661
:1031100080087480A26692E5A2A3B392E4207111A4
:10312000A26792E1A2A4B392E0A26992E1A23092D6
:10313000E0F608748020710FE55A54074480A268B5
:1031400092E5A2A1B392E4F6087480F608F608F6B8
:1031500075F007788C7E007F00E62EFEE6122F1FAA
:10316000F62FFF08D5F0F2EED333122F1FF8EFD36E
:1031700033687050788CB6FF4B056AE56A24FE50C0
:1031800014756A0220210ED2217518C075190075B8
:103190001A051216AC3071030232237892E620E34E
:1031A0005520E24520E138788DE6B6007608B64233
:1031B00072D277757B037518C0751900751A0712DE
:1031C00016AC805FE56A6014D56A1130210EC22109
:1031D0007518C0751900751A061216AC023223D282
:1031E00072788D8645D254803A788D864208D262B4
:1031F00079A07A048008788DD26179947A05D272A8
:1032000075F00FE6C4540FF755F0F5F009E6540FCA
:10321000F755F0F5F00908DAEAE5F0B40F0519778B
:10322000EEC261D293C2B475F0051204E120B20679
:103230001204E130B203D5F0F11204E12275F0037B
:103240001204C9D5F0FA1230CE75F0031204C9D5B4
:10325000F0FA122F5222204C0F30710C7518B075F5
:103260001900751A001216AC227005756E1E8002C8
:10327000D21922C298C29932201EF8309918C299E8
:10328000206005753400800EC0E0C0D075D01012EB
:103290003563D0D0D0E020980132C2982060FAC0C7
:1032A000D0C0E0E8C0E0305F05C25F754800E54F80
:1032B00024FE4003754F02E54820E712E548540715
:1032C00023245FC0E074003434C0E0E59922543F09
:1032D00023232452C0E074003433C0E0E599221562
:1032E0006D023451023451D56DFAB54E08D20F75C6
:1032F000480002345702346FB462FA023451023487
:1033000051B42AF1023451F56D24C6E56D40E6242E
:10331000F5E56D50E0056D0234517820F2156D022F
:1033200034517821F2156D0234517822F2156D0274
:1033300034517823F2156D0234517824F2156D0260
:1033400034517825F2156D0234517826F2156D024C
:103350003451023485000232F8000232FE0002339A
:103360000100023307000232DF000232DF000232C6
:10337000DF000232DF0002331A0002332200023380
:103380002A000233320002333A0002334200023391
:103390004A000232E7000232E7000232E70002325E
:1033A000E7000232E7000232E7000232E7000232B1
:1033B000E7000232E7000232E7000232E7000232A1
:1033C000E7000232E7000232E7000232E700023291
:1033D000E7000232E7000232E7000232E700023281
:1033E000E7000232E7000232E7000232E700023271
:1033F000E7000232E7000232E7000232E700023261
:10340000E7000232E7000232E7000232E700023250
:10341000E7000232E7000232E7000232E700023240
:10342000E7000232E7000232E7000232E700023230
:10343000E7000232E7000232E7000232E700023220
:10344000E7000232E7000232E7000232E70002340E
:10345000850548254EF54ED0E0F8D0E0D0D032803A
:103460000E802A802D8030803280348040803EB4AF
:103470000908754E0075480080D7B44208754E00A3
:1034800075488080CC754E0075480080CAB51EDF37
:1034900080BFB51FDA80BAF54980B6F54A80B2B56B
:1034A0004ECD754F201234AF75480080AA80D68566
:1034B0004936125DF7D260E536B44603023EE0B409
:1034C0004704125E0D22B4500D854A35125DD2C2FA
:1034D000ACC260D21722B45311854A35E54A70094F
:1034E000125DD2C2ACC260D21222B4540D854A35EC
:1034F000125DD2C2ACC260D21122B4550D854A35DC
:10350000125DD2C2ACC260D21322B4560D854A35C8
:10351000125DD2C2ACC260D21422B4570D854A35B6
:10352000125DD2C2ACC260D21522B4580D854A35A4
:10353000125DD2C2ACC260D21622B44E12854A3598
:10354000E54AB4000A125DD2C2ACC260D21822248D
:10355000BF24E64004854A3522C26022C53725379C
:10356000C53722E53424F0400EE534232482C0E040
:1035700074003435C0E022759906C260753400D2FB
:10358000B6228036803B803D803F80408045804D24
:10359000804F8058805680548052804D8057800DD7
:1035A0008015753403F59912355C053422A835E68B
:1035B00030002CE20235DF023626753700740380B6
:1035C000E4E51E80E0E51F80DC02366FE5377534E8
:1035D0000F80D21216DA123269883580C8E535803C
:1035E000C1E535A25392E080B9753403A83505359D
:1035F000E676FF80B0E535C313602714700BA22D6B
:1036000092E0B392E1440480D614700BA22E92E0B3
:10361000B392E1440880C8147008A22F92E0440CD1
:1036200080BD74FC80B9E5351470107408A26C92EA
:10363000E0A26D92E1A23092E280A41470107410A6
:10364000A22D92E0A22E92E1A22F92E2809114701C
:103650000C7418A22092E0A22192E1808214700BD7
:10366000A26E92E0A26F92E10235DFE40235DFE55F
:1036700036B441067534040235A5B4422AE53560F6
:103680000330191B53610F53620FC2AFE562B5617E
:1036900006D2AFD302369F056253620FD2AFC37515
:1036A0006E1E74420235A2B444552008F7E535C3B6
:1036B000137022B3926A122C104040203C3D303DE2
:1036C0000B205205306A348003206A2FA26A92537D
:1036D00092520236FB926A14C0E0030303540F2493
:1036E00043F8D0E0540704FA7400D333DAFD306AAB
:1036F00005FAE24A8004F4FAE25AF6E53680A5B407
:103700004B028003023794E53554F8B40812E535CE
:103710005407603714604314604714605C023577C7
:10372000B4200FE5355407605914605C14605F02E3
:103730003577B42813E535A2E09253757A0150032A
:10374000757A02E5360235A2023577751AF4C26D34
:10375000C26C755601755701805E751AF3D26D8083
:10376000EF751AF2D26CC26D755601755701C230F1
:10377000A230B392A7D26B803F751AF1D26CC26DA2
:103780008031C26EC26F8039D26EC26F8033C26E1A
:10379000D26F802DB4430FB53503755003753407D0
:1037A0007535A80235A5B44A20E5357019206D1687
:1037B000751AF0C20A12239E75181075190F121689
:1037C000ACE5360235A2023577B4450675340602FB
:1037D00035A5B4510675340C0235A5B44D0EE5354A
:1037E000121722E5365002B2E70236A4B44C067531
:1037F000340E0235A5B4460280C9B4470280C4B471
:103800004F08C256C257C25880B9B45908C2007591
:10381000340D0235A5B45A08D20075340D0235A511
:10382000023577E570C2756002D275E55BF55CC262
:1038300059206109306203023885023CA11205CD8E
:10384000122097121F247020206E08206F17123D3F
:103850001550121205A61222AC30620CE542600827
:10386000121D83700302397D75543CD550147518B0
:103870003075190085501A1216AC755003D2577561
:1038800053B4023C8C1205CDE54260F6B402061238
:103890004CFA023CA1207119201D03303E13B405DF
:1038A0001078A0B60A0B08B601028008B6030280A1
:1038B0000302395008E675F00AA4082675F00AA438
:1038C0000826C5F0703B78A1B60339201D09C0F069
:1038D000123CD0D0F0502A85F05B85F05C12059C3C
:1038E000201D0F7518C0751903855B1A1216AC02DE
:1038F0003CA17518C0751902855B1A1216AC023C02
:10390000A1023C84201D09C0F0123CBCD0F050F153
:1039100085F05B201D0E7518C0751906855B1A129F
:1039200016AC800C7518C0751905855B1A1216AC9B
:10393000125400123D02D2A2C269C2A1D26812057D
:10394000A612233AA26172625003023831023CA1EE
:10395000121FFA7025206E08206F22123D15501D8F
:103960001205A612233A3061111205CD1220977864
:1039700094797C7A05121CD460030238687554006F
:10398000755003C258C257205902C256C082C08324
:10399000123DBCD083D0825006123C40023CA1C0F4
:1039A00082C083120A19D083D0825006123C400292
:1039B0003CA1E58224CEE58334FF5013123D034041
:1039C0000E122C105006123C31023CA1023B811217
:1039D000245F5012123C31023B38123C2B023B3820
:1039E000123C25023B38206DF13039032053F1E5BC
:1039F000416058E5416009231205154003023A0968
:103A0000023A4B123C1F023B383008F7301CF430AE
:103A10004BF1A271304D01B3503130081BC0E0783A
:103A20007CE26012C3335004D0E080D712051550F9
:103A3000F7D0E0023A38D0E0C082C083125C80D078
:103A400083D0825006123C36023B38301C49125C4F
:103A50002CA2E0921AA2E1921BA271304D01B39206
:103A600005B40005200522802BB4012220051A751B
:103A700018C0751900751A091216AC204706123CB9
:103A80003B023B38123CB2800E125BA98009B402A3
:103A9000ED2005DB125BD230087930081CC0E078DD
:103AA0007BE26013C3335005D0E0023B13120515CF
:103AB00050F6D0E0023AB9D0E0207516A2719274A7
:103AC000858371858272123CAE1205B77570020251
:103AD0003CA1757000E5836571F5F0E5826572457E
:103AE000F07006123C45023B387518C07519007518
:103AF0001A0C1216AC30740C7518B0751900751AC2
:103B0000001216AC123C6A75181085711985721A6C
:103B10001216ACC2A2C269123CAAA271920AD209C0
:103B200012239E123256123C6A751810858319852D
:103B3000821A1216AC12059C123D0C5003023CA1D5
:103B4000122C1040F8D2A3C266C2A1D268D2A4C27D
:103B500067755A0012323D121DFDC082C0831223C8
:103B60003AD083D082206106206211023CA1789471
:103B7000797C7A05121CD46008023C8C121D83707B
:103B8000F8301C24E4A21A92E0A21B92E1B40305CF
:103B9000125BFE8013B40205125BA9800BB4010511
:103BA000125BD28003125B8030081CC0E07879E29F
:103BB0006013C3335005D0E0023C8C12051550F65B
:103BC000D0E0023BC7D0E0304E0FE582458360096C
:103BD000023BD9123C19023CA1B253123256305367
:103BE0001A75187085831985821A1216ACC2A3C281
:103BF00066D2A1C268D2A4C2678018751860858396
:103C00001985821A1216ACD2A3C266D2A1C268C2AA
:103C1000A4C26712059C023CA112570A023C48123A
:103C2000570A023C4812570A023C4812570A023C03
:103C30004812570A801212570A800D12570A80083C
:103C400012570A800312570A7570007571FF75725A
:103C5000FF122CBE12325675182085831985821AE0
:103C60001216AC120589122CC822207116E55B04CD
:103C7000601114656F600C7518C0751901855B1AA9
:103C80001216AC2212570A120578801512570A1222
:103C90002CBE120578122CC87570007571FF7572F4
:103CA000FFC262C261E55CF55B2212570A2212571D
:103CB0000A2212570A75F0321205E9227408F974C3
:103CC0007CF8752F0175300375319812087B8012CE
:103CD0007408F9747CF8752F0175300375319012F2
:103CE000087B7881E6085608560460141205A6126F
:103CF00022AC306209E5426005121D836002C322D6
:103D0000D32222E582249CE58334FF22E582249C91
:103D1000E58334FF22A250E58245836010E58224CA
:103D20009CE58334FF5004A24F8002A25122E58219
:103D30002582F582E5833583F583E5822582F58248
:103D4000E5833583F583E5822400F582E583345BE2
:103D5000F5837404F97400F8752F0185833085822A
:103D600031120856227881E654C0F5837882E63015
:103D7000E402240A2323543C4583F5837881E6C476
:103D8000540375F00AA4F5F0E6540F25F00303037D
:103D9000F5F053F0E085F08254034583F583788095
:103DA000E6C4540375F00AA4F5F0E6540F25F04577
:103DB00082F58222C39582E5F0958322123D2E780A
:103DC00000E2B4FF03023E3C1261CA123D65787CFA
:103DD000A68308A6827800E2F58308E2F58208E26D
:103DE000F5F008E2123DB4502B7800E2F58308E2CA
:103DF000F582787C86F008E6123DB450417802E204
:103E0000F58308E2F582787C86F008E6123DB4403E
:103E10002D023E3C7800E2F58308E2F582787C864C
:103E2000F008E6123DB440167802E2F58308E2F5A8
:103E300082787C86F008E6123DB45002C322D32279
:103E4000C5372537C53722E55424E94008D2A3C237
:103E500066D2A2C2693098EFC298E599123E40221C
:103E60003099FDC299F599123E4022C2A3C266C2A2
:103E7000A2C269C2B67537007405123E60E51E1213
:103E80003E60E51F123E60221204F91204F912048A
:103E9000F9123E6BE536123E60E537123E6030990E
:103EA000FD22120D72023EAB120D0EC0E0123E6BEF
:103EB000E536123E60D0E0123E60E537123E6030DB
:103EC00099FD221204F9123E6BE536123E60797CB0
:103ED000E7123E6009DDF9E537123E603099FD22B8
:103EE000751A00755419D21EE53E600B54F8700720
:103EF000C231A231B392A5E53F600B54F87007C2FE
:103F000032A232B392A6D2A0C28EC28CC2ADC2ABD4
:103F1000C2ACC2AF7581CD903F22C082C08375D044
:103F20000032D2AFD28C125DD2C2ACD299123E888E
:103F3000B2B5755419D298023F5FB40922F5371211
:103F40003E47B51E27123E47B51F21123E47B446D5
:103F50001B123E47AF37123E476F7010123E88D299
:103F6000B6D2A3C266D2A2C269123E47B40ACBF54A
:103F700037123E47B51EF5123E47B51FEF123E47BA
:103F8000F536B46D0302400FB46E03024028B46FDF
:103F90000302405FB470030240ACB471030240C03E
:103FA000B473030240D1B474030240D3B475030266
:103FB00040E7B476030240FFB47703024113B478BC
:103FC00003024127B47903024148B47A03024164F1
:103FD000B46C03024178B46B0302419AB46A0302E1
:103FE00041D5B469030241F1B46803024233B467B6
:103FF0000302424BB46603024266B4650302432ADD
:10400000B46403024AA2B46103024AFD023F5FAFF7
:1040100037123E476F70F5123E88D2B675F01E1209
:1040200004C9D5F0FA025F6A123E47FD1424E0404D
:104030002B123E472400FC7B00123E47FEAF371296
:104040003E476F70178EF0EDF9747CF88B2F8C3033
:1040500085F03112087B123EC3755419023F5F127E
:104060003E47FD1454E070F4123E472400FC2471D6
:1040700040EA7B02123E47FEEDFA787C123E47F69C
:1040800008DAF9AF37123E476F70D1C2A3C266C2D9
:10409000A2C2698EF0EDF9747CF88B2F8C3085F01C
:1040A000311207D0123E9175541980B0AF37123ECD
:1040B000476F70A8120B30123E88755419023F5F8B
:1040C000AF37123E476F7009123EA8755419023F70
:1040D0005F8089123E47FD1424E04048123E472489
:1040E00000FC7B01024039123E47FD1454E070345D
:1040F000123E472400FC2425402A7B03024074AF73
:1041000037123E476F701D024124123E91755419BB
:10411000023F5FAF37123E476F7009123EA27554DF
:1041200019023F5F02405C79207D07123E47F30988
:10413000DDFCAF37123E476F70EA1252DF40E512E6
:1041400061AB123E91023F5FAF37123E476F70D4B2
:104150001261CA1204F9123E6BE536123E60121566
:1041600041023F5FAF37123E476F70661211631214
:104170003E88755419023F5F123E47FE123E47FDCE
:10418000123E47FCAF37123E476F7046120A964008
:1041900041123E88755419023F5F123E47FE123E9F
:1041A00047FDAF37123E476F7028120A671204F9B5
:1041B0001204F9123E6BE536123E60EE123E60EDDF
:1041C000123E60EC123E60E537123E603099FD020F
:1041D0003F5F02405CAF37123E476F70F51204F943
:1041E0001204F9123E6BE536123E601215D1023F01
:1041F0005FAF37123E476F70D9120D06600274012F
:10420000C0E0120D6A60027402D0F045F0700A122C
:104210000B7B121919121163E4C0E0123E6BE536F4
:10422000123E60D0E0123E60E537123E603099FDEC
:10423000023F5F123E47FD1454E07027123E4724B0
:1042400000FC2471401D7B00024074123E47FD14A7
:1042500054E0700F123E472400FC242540057B01EA
:1042600002407402405CAF37123E476F70F5120493
:10427000F91204F9123E6BE536123E607401123EEB
:1042800060744E123E60746E123E607448123E605E
:104290007435123E607400123E60748D123E60747C
:1042A00020123E6074DA123E607400123E60740F99
:1042B000123E6074A0123E607480123E6074001260
:1042C0003E607400123E607420123E607400123E24
:1042D000607400123E607400123E607400123E6012
:1042E0007400123E607400123E607400123E6074EE
:1042F00000123E607400123E607400123E60740052
:10430000123E607400123E607400123E607400122F
:104310003E607400123E607400123E60E537123E4B
:10432000603099FD023F5F02405C123E47F5831208
:104330003E47F5822460E58334F040EB12461312C9
:104340003E47FD1454E070DF7800123E47F208DD6E
:10435000F9AF37123E476F70CE123E8875F00512E6
:1043600004C9D5F0FA123E91751A013008B9300728
:10437000B612468712466D124621121DFD789479B9
:10438000007A0A75F00FE3540FF652F00809DAF6D6
:1043900043F0F0E5F0047894797C7A05121CD4603F
:1043A0000B1244425006751A0402432712466D123E
:1043B0004621121DFD78A0790A7A0675F00FE354A4
:1043C0000FF652F00809DAF643F0F0E5F00478A0B1
:1043D00079817A03121CD4600B1244E05006751ADE
:1043E0000602432712466D1246D0751A65023F5FDA
:1043F000C0E07830E583F208E582F2D0E022C0E048
:104400007832E583F208E582F2D0E022C0E078302D
:10441000E2F58308E2F582D0E022C0E07832E2F5EE
:104420008308E2F582D0E022E5822400F582E5836C
:10443000341BF58322E5822400F582E583343BF5C5
:104440008322124621AB83AC82901B00C08379008B
:10445000752F038583307531009000361207851261
:1044600008F61207851209549000367A80E0A3F509
:10447000F0E0A36C7005E5F06B6017DAF0D083050F
:1044800083740024C0E58334C550C1740512458F80
:10449000D322D083EA2AF5F0E4C395F0F5821243E3
:1044A000F0789479007A0A75F00FE3540FF652F021
:1044B0000809DAF643F0F0E5F004600C121F2970E9
:1044C0000A740612458FD322121F29E5822582F530
:1044D00082E5833583F5831244281243FE0248A700
:1044E000124621AB83AC82903B00C0837900752FCC
:1044F000038583307531009000361207851208F667
:104500001207851209549000367A80E0A3F5F0E096
:10451000A36C7005E5F06B6017DAF0D08305837447
:104520000024C0E58334A550C1740512458FD32201
:10453000D083EA2AF5F0E4C395F0F5821243F078CF
:10454000A0790A7A0675F00FE3540FF652F00809C5
:10455000DAF643F0F0E5F004601D12200A701BABA0
:1045600083AC82124621EBB58306ECB58202C322EE
:10457000740412458FD32212200AE5822582F58227
:10458000E5833583F5831244351243FE0248A7F5CF
:104590001A22C082C083E5831252DED083D082C04B
:1045A00082C083E5821252DED083D08222C082C0D4
:1045B000837F00E58224F0C0E0E58334D8C0E0507A
:1045C00007D083D0820F80EBD0E0D0E07F00E5827F
:1045D0002418C0E0E58334FCC0E05007D083D082CB
:1045E0000F80EBD0E0D0E07F00E582249CC0E0E5C6
:1045F0008334FFC0E05007D083D0820F80EBD0E03F
:10460000D0E0E58275F00A84C0F0F5F0D0F0D083F8
:10461000D08222C0E07834E583F208E582F2D0E06F
:1046200022C0E07834E2F58308E2F582D0E0227817
:1046300081E61252DE7882E61252DE7883E612526A
:10464000DE78A0E61252DE78A1E61252DE78A2E60B
:104650001252DE78A3E61252DE78A4E61252DE7819
:10466000A5E61252DE120E0422120E04227400126B
:104670003E607400123E607400123E607400123E90
:10468000607400123E602275831B75821B75F040BA
:10469000C0F0C082C083752F018583307531001250
:1046A00007851208F6D083D082C082C083752F039D
:1046B0008582307531001207851209BCD083D08203
:1046C00005830582D0F0D5F0C77532FF7533FF2220
:1046D0007401F97418F8752F0075300075310012E7
:1046E000087B7401F97419F8752F017530D975318B
:1046F000FF12087BAC18124621E5822420F582E5E2
:1047000083347DF583C082C0837401F97441F875E8
:104710002F0085833085823112087BD083D082744C
:1047200001F97410F8752F008583308582311207E6
:104730009F7810E2F5F0E5182541C395F0F51812C1
:104740004621E58275F008A42420F582500205F088
:10475000A8F0E58375F008A4282400F5837408F90F
:10476000747CF8752F0085833085823112087B7840
:104770007CE5187A082608DAFCF518789479007A2E
:104780000A75F00FE3540FF652F00809DAF643F019
:10479000F0E5F0041251ED78A0790A7A0675F00F71
:1047A000E3540FF652F00809DAF643F0F0E5F004AE
:1047B0001251F57408F9747CF8752F0085833085E3
:1047C00082311207D0787CE5187A08C39608DAFBA4
:1047D000F518124621C3E58233F582E58333F5836C
:1047E000C3E58233F582E58333F583E5822400F562
:1047F00082E583245BF583C082C0837404F9747CF2
:10480000F8752F0185833085823112087BD083D0E3
:10481000827404F97412F8752F0185833085823112
:1048200012079F787C7912E5197A0426F5F0E3C522
:10483000F0C395F00809DAF3F5197401F97418F862
:10484000752F007530007531001207D07401F974AE
:1048500019F8752F017530D97531FF1207D075839E
:104860001B75821B75F040C0F0C082C083752F039A
:104870008583307531001207851208F6D083D08207
:10488000C082C083752F0185823075310012078583
:104890001209BCD083D08205830582D0F0D5F0C741
:1048A0007532FF7533FF2212441AE5828583F012B8
:1048B000440CC39582C0E0E5F09583D0F045F070DC
:1048C00002C32250030249C212441AC0E0C3E58267
:1048D00024FEF582E58334FFF583D0E01243FEE544
:1048E000828583F012440CB58207E5F0B58302C3DC
:1048F0002212440CAF8312441AEFB58310AE82909B
:104900000034787CE0F6A308E0F60249257EFE8FAD
:104910008305837402F9747CF8752F0385833075E1
:10492000310012087B7900752F038F3075310090AC
:1049300000361207851208F61207851209548F8374
:1049400075820012440C7D00E5836F7002AD82ED2C
:104950002436F58275830050020583C3EE9D20E066
:104960005A03FCC082C083A3A3E0FAA3E0FBD08378
:10497000D082EAF0A3EBF0A3DCE9EE2436F58275F1
:10498000830050020583787CE6F0A308E6F0790006
:10499000752F038F3075310090003612078512098C
:1049A000A81207851209BC852F3285303312441AAC
:1049B000EFB58303024A960F0248F6740812458F3A
:1049C000D32212440CAF8312441AEFB58310AE8287
:1049D000900034787CE0F6A308E0F60249F67E0009
:1049E0008F8315837402F9747CF8752F03858330E7
:1049F0007531FE12087B7900752F038F30753100F9
:104A00009000361207851208F61207851209541213
:104A1000440C7DFEE5836F7002AD82ED2436F58295
:104A200075830050020583C3ED9E20E06B03FCC03C
:104A3000E0C3E58224FEF582E58334FFF583D0E010
:104A4000C082C083E0FAA3E0FBA3EAF0A3EBF0D0BE
:104A500083D082DCDAEE2436F582758300500205BD
:104A600083787CE6F0A308E6F07900752F038F3099
:104A70007531009000361207851209A812078512B9
:104A800009BC852F3285303312441AEFB5830302F7
:104A90004A961F0249C7C322740912458FD32202C6
:104AA000405C123E47F583123E47F582AF37123E17
:104AB000476F70EBC01EC01F85831E85821F121CAE
:104AC000597401F9747CF8752F0075300075310048
:104AD00012087B787CE6C3951EC3951FD01FD01E9D
:104AE000251E251FF67401F9747CF8752F007530AA
:104AF000007531001207D0123E88023F5F123E4718
:104B0000F583AF37123E476F70951204F91204F91E
:104B10001204F9123E6BE536123E607400123E60DC
:104B2000E51A123E607400123E607400123E60741A
:104B300000123E607400123E60E537123E6030990C
:104B4000FD023F5F904B4CC082C083327581CD75B2
:104B5000D000025F6AC082C083E5822420F582E52E
:104B600083347DF5837401F97441F8752F008583D2
:104B7000308582311207D0D083D082C082C083E5D5
:104B80008275F008A42420F582500205F0A8F0E513
:104B90008375F008A4282400F5837404F9747CF864
:104BA000752F008583308582311207D0A3A3A3A37C
:104BB000747C2404F5F07404F9E5F0F8752F008591
:104BC00083308582311207D0D083D082C20722126F
:104BD0000D0EC0E07401F9747CF8752F007530007B
:104BE00075310012087B787CE6D0F0C395F0F6743E
:104BF00001F9747CF8752F007530007531001207CB
:104C0000D022120578C2AF80FE30081CC0E078794F
:104C1000E26013C3335005D0E0024CA012051550DA
:104C2000F6D0E0024C28D0E0D2A3C266C2A1D2687E
:104C3000D2A4C2671205A612233A20610620623070
:104C4000024CA01205DF121F247055123D0C40507B
:104C5000206E08206F4C123D1550471205A61222F7
:104C6000AC30623CE5426038121D837033024CA2C6
:104C7000E542602C1205DF121FFA7024123D0C4031
:104C80001F206E08206F1B123D1550161205A6122C
:104C9000233A30610B7894797C7A05121CD4600237
:104CA000D322304E18E58245836012E54160092326
:104CB0001205154003024CBB024CBD80E3B253C346
:104CC00012325630531A75187085831985821A125C
:104CD00016ACC2A3C266D2A1C268D2A4C2678018B1
:104CE00075186085831985821A1216ACD2A3C26624
:104CF000D2A1C268C2A4C267C32278A0E6B40A17D0
:104D000008E6B40545122C104009124C0940041263
:104D1000059C221205782275F00AA4F5F008E62514
:104D2000F0B46326D2A3C266C2A2D269C2A1D2687D
:104D3000D2A4C267C0E01205A612233A9000001266
:104D40001DFD20610920622BD0E01205782212059A
:104D5000DF7894797C7A05121CD470EC30503A12CA
:104D600005A61222AC3062E01205DF121D8370D856
:104D7000024D991205DFE54260CE121D8370C930E5
:104D800050171205A612233A3061BD1205DF789440
:104D9000797C7A05121CD470AF1205A6D0E0B40B52
:104DA0000812505E4024024ED3B40C0812509F40AB
:104DB00019024ED3B40D081250CA400E024ED3B49D
:104DC0000E0B1250D94003024EE2024ECFB40F2810
:104DD0001261CA12524B401DF824DC4018E878805A
:104DE000F612524B400FF824A0400AE8787FF612E2
:104DF00061AB024ED3024ECFB410028003024E6F5D
:104E00001261CA1222A82054061222A83054E612B7
:104E100016F3C0E0D0E0F824F640DAE8131354C0EB
:104E20007881F612524B40CD60CBF824ED40C6E8B5
:104E30007882F612524B40346032F824CE402DE88E
:104E4000788146F61222A82054061222A830541C5B
:104E50001216F3C0E0D0E0F824F94010E813131361
:104E600054C0788246F61261AB024ED3024ECFB4E4
:104E7000111512170BB4010C12170BB407061250C0
:104E8000E8024ED3024ECFB413202038F712233A53
:104E900020620B3061EE121DA57034024C02E54217
:104EA000602D121DC17028024C02B4632212170B30
:104EB000B40A1C12170BF57790017D700390018ADC
:104EC00075F0641204C9D5F0FA024ED3024ECF1227
:104ED000057822124BCF7518C0751900751A0A1281
:104EE00016AC12059C22754100787C75F00876FF9F
:104EF00008D5F0FA22EFC0E0C25A789979817A0693
:104F0000EA30E004E6088002E6C4540FFFEA30E02D
:104F100004E7098002E7C4540FB40F10BF0F10EA72
:104F20006406600B205A1ED0E0FFE422BF0F06D0BB
:104F3000E0FF740122205AF7F5F08F476F6002D22C
:104F40005ADABD80DFE5F0C395475002F4041460DF
:104F5000D6B408DB80D17894797C7A057401B6FFE9
:104F600002800FB7FF02800AE66770060809DAF8C8
:104F7000E422740122124F80E58245837001D3221E
:104F80008005D0E0024FD112170BC0E024F640F2AA
:104F9000D0E075F00AA4F5828005D0E0024FD1126E
:104FA000170BC0E024F640F2D0E0258275F00AA489
:104FB000F58285F0838005D0E0024FD112170BC037
:104FC000E024F640F2D0E02582F58250020583C34A
:104FD00022D322C082C083900000121E59124F5665
:104FE000701AE5828583F0D083D082B5821FC5F028
:104FF000B5831AC082C083F58385F082A3E583B4AC
:105000000FD8E582B4A0D3D083D082C322D322C0EC
:1050100082C083900000121E59124EF5701AE5826C
:105020008583F0D083D082B5821FC5F0B5831AC0C6
:1050300082C083F58385F082A3E583B40FD8E5822F
:10504000B4A0D3D083D082C322D32212233A3061BA
:10505000311251ED121DD7C3229000008008124F6B
:1050600075401F1205A612233A3061161205DF1291
:105070001DFD1251ED124FD34008754100124B55E2
:10508000C322D3221222AC3062F8E54224FD24FC74
:1050900040F01251F5121DEAC32290000080081260
:1050A0004F7540DE1205A61222AC3062D5121DFDEE
:1050B0001251F5E542600B24FD24FC40C512500F4F
:1050C00040C0754100124B55C322124F7540081263
:1050D0004EE6124B55C322D322124F754008121DC3
:1050E000FD125137B322D322C20790002874D8F999
:1050F00074FFF8752F01858330858231120CBE75DF
:10510000830175F01E752F00858330753100C0F066
:10511000C083120785120C9ED0830583D0F0D5F092
:10512000E4907D007420F974FFF8752F01858330B9
:10513000858231120CBE22787CE6080808080856E1
:10514000B4FF02D322C322751E30751F30C271C254
:105150007275F005C0F0D2A3C266C2A2D269D2A114
:10516000C268D2A4C267124EE612233AD0F0206180
:1051700009206206D5F0DD0251BE12520D403F12E9
:10518000059C7881E6B4FF05C32275F005C0F012D6
:10519000233AD0F0206206D5F0F30251BEE542B4C6
:1051A000021C78A0E624F6401508E624F6400F78A5
:1051B000A0E62430F51E08E62430F51FC3221205B0
:1051C00078D3227546008003754601C25512233AF2
:1051D00020620B30610A0546E54624F550EFD322E4
:1051E000E5466007D255B40A027400C32278947968
:1051F0007C7A05800678A079817A03E608540FC48A
:10520000F5F0E608540F45F0F709DAEF2220613196
:10521000306236E542600624FD24FC402C1251F534
:105220001205A675F005C0F0122336D0F0206111EA
:10523000205406D5F0F00252491216F3B40B0A803E
:10524000031251ED754100C322D3221222A820542B
:10525000061222A830542B1216F3C0E0D0E0F82436
:10526000F6401F1222A82054061222A8305413120E
:1052700016F3C0E0D0E0F5F024F64006E8C445F0AF
:10528000C322D32212529475F0641204C9D5F0FAE5
:1052900012054B2275F03C1205E9C2A075F03C12D4
:1052A00005E9D2A075F0141205E9C2A075F03C1210
:1052B00005E9D2A075F0141205E9C2A075F0141228
:1052C00005E9D2A075F0141205E9C2A075F0141218
:1052D00005E9D2A02275F00A84C0F0D0F02222782D
:1052E00025E254C07078E275F00A84C445F0787EF7
:1052F000F67824E254C07066E275F00A84C445F082
:10530000787FF67823E254E07054E275F00A84C4A2
:1053100045F07880F67822E2604454E07040E2750F
:10532000F00A84C445F0C0E07820E2030354C0D002
:10533000F045F07881F67821E2602354F0701FE2A6
:1053400075F00A84C445F0C0E07826E254F8700E87
:10535000E2C42354E0D0F045F07882F6C322D32291
:1053600090000075F019C0F07402F9747CF8752F84
:105370000185833085823112087B787DB6FF0280FB
:105380000E18E55B300805B4FF02E56F666011E5B5
:10539000822410F58250020583D0F0D5F0C8C322D4
:1053A000D0F0A3D32230084DE58224FFF582E583B7
:1053B00034FFF58375F019E5822480E58334FE50CF
:1053C00005900000800AE5822410F58250020583D2
:1053D000C0F07402F9747CF8752F018583308582E2
:1053E0003112087B787DB6FF02800518E6B55B07B1
:1053F000D0F0D5F0C2C322D0F0A3D3222202542B86
:10540000300FFAC20F1252DF40F31261AB02542E7A
:105410007822E21252D57821E21252D57823E21294
:1054200052D57824E21252D50254521261CA7881C0
:10543000E6C45403E6540F7882E6C45401E6540FE0
:105440007880E6C4540FE6540F787FE6C4540FE624
:10545000540F30080A12536050051253FC80031297
:10546000546322E55BB4FF069002CA0254A2B40062
:105470000690010A0254A2B410069001130254A22D
:10548000B4110690011C0254A2B420069001260219
:1054900054A2E55B75F06484C0F0D0E01252D59060
:1054A000015222201C0122758205125B10600F75CB
:1054B000F0021204C9D5F0FAD582EF125B127475AE
:1054C00078431205FA5015207614D276125B1275C5
:1054D00018C0751900751A0D1216AC22C276126129
:1054E000CA203F0420402E227880E6543FF5F07910
:1054F0003FE365F0701C09E3787F66701520411169
:10550000D241125B127518C0751900751A0D12166A
:10551000AC2230402A7880E6543FF5F07941E365CB
:10552000F0701C09E3787F667015204111D241129A
:105530005B127518C0751900751A0D1216AC22C2CF
:105540004122C2AC1216DA6024F51888191211D65D
:1055500053610F53620FC2AFE562B56106D2AFD39C
:1055600002556B056253620FD2AFC380D7D2AC2213
:105570007E007F6490000075F000E49325F0F5F064
:10558000A3C3E5829EE5839F40F0E5F0700122E52C
:10559000F0C0E0E5831252DEE5821252DED0E01266
:1055A00052DEC2ADC2ACD21E12056320B7FA75F04E
:1055B000C81204C9D5F0FA30B7FD75F0C81204C995
:1055C000D5F0FA125DD22275F0641209CF20E512EF
:1055D00030E30F221204E1B2B51204E1B2B5D5F006
:1055E000F322C2AFB2B51204E1B2B51204E1D5F0B4
:1055F000D9C2A075F0321255D4D2A075F03212552E
:10560000D4C2A075F0321255D4D2A075F032125522
:10561000D475F0961255D480D82230083C740078A6
:105620005312060940337F087E00747878431205D0
:10563000FACE13CE05E0DFF4201F0E74007863125B
:1056400006095005EE655D60108E5D8E5B7518C0B5
:10565000751904855B1A1216AC22C2AF7518107545
:10566000190FF51A1216ACD2AF223008097401785E
:1056700053120609500122747778431205FAE49216
:10568000E0C0E0747678431205FAD0E033FE201FC4
:105690000E740178631206095005EE655E60D78EC0
:1056A0005EEE20E10630E02E0256F330E017A26DE8
:1056B000726C50C2C26DC26C75560175570174F898
:1056C00012565A80B1D26DC26C755601755701746D
:1056D000F712565A80A0206C9DD26CC26D7556018F
:1056E000755701C230A230B392A7D26B74F612562E
:1056F0005A8083A230826C40F8D26CC26DC20A120A
:10570000239E74F512565A025676C082C083D08307
:10571000D082222222C2A075F0141204C9D5F0FA58
:10572000D2A075F0141204C9D5F0FA22C2A075F007
:105730003C1204C9D5F0FAD2A075F0141204C9D5F0
:10574000F0FA2212571512571512572C12571575C9
:10575000F0641204C9D5F0FA2212572C1257151210
:10576000571512571575F0641204C9D5F0FA223096
:105770005309C2A3C266D2A4C26722D2A3C266C220
:10578000A4C2672230084930081CC0E0787AE26081
:1057900013C3335005D0E00257BC12051550F6D0A4
:1057A000E00257A6D0E0D26E201F032070227518A9
:1057B000C0751900751A0F1216AC8014C26E201F26
:1057C0000330700C7518C0751900751A101216ACDC
:1057D000A26E927022094300A00954009F0966003E
:1057E0009E0977009D0989009C099B009B09AD00DB
:1057F0009A09BF009909D2009809E4009709F700B7
:10580000960A0A00950A1D00940A3000930A430084
:10581000920A5700910A6B00900A7F008F0A93004A
:105820008E0AA7008D0ABB008C0AD1008B0AE70004
:105830008A0AFE00890B1400880B2B00870B43009B
:10584000860B5C00850B7500840B8E00830BA70014
:10585000820BC100810BDB00800BF6007F0C100077
:105860007E0C2B007D0C47007C0C64007B0C8100BF
:105870007A0C9E00790CBB00780CDB00770CFB00E7
:10588000760D1B00750D3B00740D5B00730D7D00E4
:10589000720D9F00710DC200700DE4006F0E0700C5
:1058A0006E0E2C006D0E51006C0E76006B0E9B0080
:1058B0006A0EC100690EE900680F1100670F390018
:1058C000660F6100650F8900640FB300630FDE008F
:1058D000621009006110340060105F005F7F429029
:1058E00057D5E493A3F5F0E493A3C3958BE5F09526
:1058F0008D5015A3A3DFEBE58224FFF582E5833409
:10590000FFF583E49314800BA3E493BF4205905703
:10591000D58010C0E0E58224F9F582E58334FFF5F7
:1059200083D0E02290003AE0A28733F02290003B3F
:105930007400F090003A7455F090003C74FFF090C1
:10594000003E7405F090003D7412F0D28122D286A0
:10595000A2A4C0D0D2A475F000D5F0FDD5F0FDC250
:105960008E53890F438910758B00758D00C28FC2CD
:10597000AFC2A4D28E208603308FFAC28E308F063B
:10598000758BFF758DFFD2AFD0D092A422F024FD8D
:105990004005308102C2812290003EE0D5E0EE74E5
:1059A00042F012594ED281E58B2499E58D34F240B4
:1059B00014E58B24E1E58D34F3400EE58B249CE562
:1059C0008D34FF400874158006741180027412FE35
:1059D00090003DE06E6010EEF020030B7518C0756E
:1059E00019008E1A1216AC22125924603604603344
:1059F00090003CE020E010D2E0F090003BE070042A
:105A00007405F022E4F02290003BE0602914F0706D
:105A1000252002227518C0751900751A141216ACCB
:105A2000025A3690003CE030E00DC2E0F090003BBE
:105A3000E070D1743CF02290003BE060F914F0700B
:105A4000F52002F27518C0751900751A131216ACFC
:105A500080E41259981259E822C2B612594E1258CF
:105A6000DD7537007403123E60E51E123E60E51FCF
:105A7000123E60744E123E60740C123E607400124E
:105A80003E60740A123E60C082C083A3A3A3E49365
:105A900075F064A4C0E0E5F0123E60D0E0123E6014
:105AA000A3A3A3A3E49375F064A4C0E0E5F0123EC1
:105AB00060D0E0123E60D083D082E493123E60A3B7
:105AC000E493123E60A3A3A3E493123E60A3E49385
:105AD000123E60E58D123E60E58B123E60E53712A6
:105AE0003E603099FD221208C6C28474541208E048
:105AF000E41208A01208B3F5F06448256733F5678F
:105B0000E5F02568B2E003F568D9E9D284222222C3
:105B1000E4227583DD75F010752F038583307531B0
:105B200000C083C0F0120785120C9ED0F0D0830510
:105B300083D5F0E47532FF7533FF125B0F22025BF1
:105B400071C082C083758205C082125B10D08260F2
:105B50001CC2A075F00F1204C9D5F0FAD2A075F0DE
:105B6000051204C9D5F0FAD582DE125B12D083D0BB
:105B700082E5822400C0E0E58334DDF8D0E0C32272
:105B8000125B41C082C083F5828883787C76007482
:105B900001F9747CF8752F038583308582311207F3
:105BA000D0D083D082125B0F22125B41C082C083AF
:105BB000F5828883787C76027401F9747CF8752FFD
:105BC000038583308582311207D0D083D082125B67
:105BD0000F22125B41125B41C082C083F582888331
:105BE000787C76017401F9747CF8752F0385833015
:105BF0008582311207D0D083D082125B0F22125BD4
:105C000041C082C083F5828883787C76037401F971
:105C1000747CF8752F038583308582311207D0D0CC
:105C200083D082125B0F22125B3E8003125B41C065
:105C300082C083F58288837401F9747CF8752F0320
:105C400085833085823112087B787CE6B40102803E
:105C50000CB402028007B4030280027400D083D027
:105C600082221208C6C28474541208E0E41208A00A
:105C70001208B3B402057567018002D9F3D28422F9
:105C80007567007583DD75F00F752F03858330759B
:105C90003100C083C0F01207851208F6120785791B
:105CA00000125C62D0F0D0830583E5677026D5F0E2
:105CB000D8752F038583307531001207851208F6D9
:105CC00012078579A0125C627532FF7533FFE567B4
:105CD0007002D322C322C28C758A45758C5DD28C2A
:105CE000B20120010132C0D0C0E0C0F075D008D2AE
:105CF00065201E04E5556002B2B51216F2125DB3BE
:105D0000051DE51D20E03920E136201E3A206905F9
:105D1000A230B392A2E51D30E203122CD2E51D544D
:105D20001F7013E4B55628B55147B55356B56E5E8E
:105D3000B57B60B55464E4B55545B5526BB54F6C51
:105D4000D0F0D0E0D0D032E51D541F60E680F130B5
:105D50004A0CE55724C24003D557CC75573CD5565D
:105D6000C6C209206CC1C230A230B392A7D26B80E8
:105D7000B6D551B6C2097553B4D258D25B80AB15B3
:105D80005580B7D553A7C256C257C258809FD56E0B
:105D90009F809DD57B9DC2778099D554997550037E
:105DA000301E03024B44808515528091D54F91D20D
:105DB0005F808DE51DA2E330660292A330690292F6
:105DC000A230680292A122C2B6206002D2B6125D51
:105DD000D23275C800C2ADC2AC75CBFF75CA98751A
:105DE000CDFF75CC98759853C298C299D2ACC2BCFD
:105DF00075C8347599062275C800C2ACC2AD7598D5
:105E00000075CC2B75CDEBD2AD75C8042275C800DA
:105E1000C2ACC2AD759800E58A242BF5CC540F6551
:105E20008C24EBF5CDD2AD75C804227580FF75903A
:105E3000FF75A0FF758F011209DCD21ED2A0755626
:105E400000755700C230A230B392A7C231A231B35D
:105E500092A5C232A232B392A6E4F541784375F01E
:105E600010F2D5F0FCC26CC26DC26EC26FC22DC200
:105E70002EC22FC254C256C257C258755301755410
:105E800000C25BD25FC260D265C217C211C212C229
:105E900013C214C241C215C216756C01C220C221C0
:105EA000754F10E4F548F549F54AF534F536751E99
:105EB00000751F80753E07753F00E4F551F559F5F3
:105EC00058F561F562F54475430F75450F751D046E
:105ED00074377836F27837F27838F2D227D228D26F
:105EE00029D23474377839F275500375520178A885
:105EF0007A0576FF08DAFBC20F7820E47A07F20809
:105F0000DAFCC210755BFF855B5DC219C208C24333
:105F1000756E1E757000C275C20DC20EC209C20A2E
:105F2000C20BC271C2721218637555FAB2B57532DE
:105F3000FF7533FF757700D276757A00782F740A73
:105F4000F2D20412592DC277757B01758901758AC9
:105F50003E758C5DC2B9D2A9D28CD2B6125DD2D2B6
:105F6000AFD293C2B4D2B2B2B522C21E755A037573
:105F7000F0031204C9D5F0FAC271C2721230CE75A4
:105F80005A0375F0031204C9D5F0FAC271C2721235
:105F90002F52C2AF020000D6435243206C696E6993
:105FA00061203300D7435244206C696E696120340C
:105FB00000C2AF7555FAB2B51204E1B2B51204E1F0
:105FC000B2B5D2A07581CD75D000125E2B12570AE2
:105FD000125570125B121220AF7555FA1210D4755B
:105FE0005A0312323D1205B0751880751904751ADE
:105FF0006E1216ACD21F30080F120F6C12561A1206
:10600000566A1254A3125784D2B7D2AFC21EC21F0F
:1060100000000020B7091204E120B7030220C930B4
:106020000815304303120F6C30080C12561A125622
:106030006A1254A3125784E5706003D57008125A8F
:1060400052125400800CD2A3C266C2A1D268D2A45C
:10605000C267E56E7006304203125542C269D2A192
:10606000C26812576FC271C272D26B12233A206299
:10607000052061028017303A0930570612570A028C
:106080006085123823782FE215E0F27008782F74BB
:1060900014F202600880910074A212612CE812616F
:1060A00067E912616712619E2274A212612CE812E4
:1060B0006167E712616709D582F812619E2274A2B6
:1060C00012612CE812616774A312612C126187F7C8
:1060D00009D5820412619E22C296D297000000C2A6
:1060E0009780E974A212612CE81261671260F022B5
:1060F00074A312612C126187F912619E2274A27A34
:1061000008C296000000C297335005D29602611271
:10611000C296D297000000C297DAEDD29600D297CD
:10612000000000309604C297C322D3227A08D29688
:10613000D2970000000000000000000000000000F6
:106140000000C296000000C297335005D29602614B
:1061500053C296D297000000C297DAEDD29600D2D1
:1061600097000000C297227A08335005D296026148
:1061700073C296D297000000C297DAEDD29600D291
:1061800097000000C297227A08D296C297000000BA
:1061900000D297C3309601B333DAF0C29722C29689
:1061A000000000D297000000D29622787C7600088A
:1061B00076007880E6543FF67800797CC08275825C
:1061C000071260A9D0821204C9227802797EC082A7
:1061D0007582051260BED082227882E603C454071D
:1061E00075F018A4C0E07880E6C4540375F00AA4E2
:1061F000F5F0E6540F25F0D0F025F075F03CA4C082
:10620000F0C0E0787FE6C4540775F00AA4F5F0E624
:10621000540F25F0D0F025F0F5F0D0E03400C5F0B3
:10622000220000000000000000000000000000004C
:10623000000000000000000000000000000000005E
:10624000000000000000000000000000000000004E
:10625000000000000000000000000000000000003E
:10626000000000000000000000000000000000002E
:10627000000000000000000000000000000000001E
:10628000000000000000000000000000000000000E
:1062900000000000000000000000000000000000FE
:1062A00000000000000000000000000000000000EE
:1062B00000000000000000000000000000000000DE
:1062C00000000000000000000000000000000000CE
:1062D00000000000000000000000000000000000BE
:1062E00000000000000000000000000000000000AE
:1062F000000000000000000000000000000000009E
:10630000000000000000000000000000000000008D
:10631000000000000000000000000000000000007D
:10632000000000000000000000000000000000006D
:10633000000000000000000000000000000000005D
:10634000000000000000000000000000000000004D
:10635000000000000000000000000000000000003D
:10636000000000000000000000000000000000002D
:10637000000000000000000000000000000000001D
:10638000000000000000000000000000000000000D
:1063900000000000000000000000000000000000FD
:1063A00000000000000000000000000000000000ED
:1063B00000000000000000000000000000000000DD
:1063C000000000000000000000000000000050522B
:1063D000343032207665722E3131302E35204864CB
:1063E000773A482034303030752032392D30352D11
:1063F00030342031323A343220204352433D00B70A
:00000001FF
:0300000306028072
